:100000009529FF3FFF3FFF3FDF00030E8301A6005E
:100010000408A5000A08A7008A015208B000510888
:10002000AF005008AE00003005190130D100510872
:10003000003A031D1F288B120130A000A1012208E5
:10004000003A031D6F2801300505D1005108003A20
:10005000FF30031D0030D200003085180130D10080
:100060005108013AFF30031D0030D00050085205FE
:10007000D1005108003A031949288B12230824069D
:10008000031D45280130A3004628A30A2308A10028
:10009000A001003085180130D1005108003AFF302E
:1000A000031D0030D20001300505D1005108013A8E
:1000B000FF30031D0030D00050085205D100510818
:1000C000003A03196F288B122308013A031D6B288D
:1000D0002408A3006C28A3032308A100A0010B118E
:1000E0003008D2002F08D1002E08D00027088A003F
:1000F00025088400260E8300DF0E5F0E0900003005
:10010000031383169C180130D1005108013A031DD6
:100110008B2800007F282C089B002D089A007F3038
:100120001C05D00050089C00043050049C008B1328
:1001300055309D00AA309D009C148B171C1108009F
:10014000031383122A0884000008AB002B08013A2D
:10015000031DC02887018230DB00FF30DA00DB0B93
:10016000B228B528DA0BB228AF288730DA00DA0BCC
:10017000B72800008716AC010130AD007F202E2982
:10018000031383162B08023A031DDD28831287010F
:100190008230DB00FF30DA00DB0BCF28D228DA0B0D
:1001A000CF28CC288730DA00DA0BD42800000716D5
:1001B000AC010230AD007F202E292B08033A031D2D
:1001C000F828831287018230DB00FF30DA00DB0B76
:1001D000EA28ED28DA0BEA28E7288730DA00DA0B7C
:1001E000EF2800008715AC010330AD007F202E29D9
:1001F0002B08043A031D1329831287018230DB0088
:10020000FF30DA00DB0B05290829DA0B0529022962
:100210008730DA00DA0B0A2900000714AC01043039
:10022000AD007F202E292B08053A031D2E298312AD
:1002300087018230DB00FF30DA00DB0B2029232925
:10024000DA0B20291D298730DA00DA0B2529000076
:100250008714AC010530AD007F202E290800031360
:100260008312280883169B009C139C131C14000007
:1002700000001A08A9002908D00008000030031364
:100280008312851A0130D1005108013A031D562905
:100290000030051A0130D1005108013A031D5329DD
:1002A0000230A80055290430A80063290030051A3F
:1002B0000130D1005108013A031D61290330A80023
:1002C00063290530A8002808D00008000313831212
:1002D0002208003A031D852987018230DB00FF30A8
:1002E000DA00DB0B74297729DA0B7429712987303E
:1002F000DA00DA0B7929000007150130A20001307D
:10030000AC000130AD007F2094290313831622082E
:10031000013A031D94292330AA00A020A201013034
:10032000AC00AD017F20942908000730031383122D
:1003300099003730831695003730850087010230E9
:100340008100073083128100A101A001A201A80150
:100350002F215008A3003E215008A400230850027A
:10036000FF3003180030D1002308003AFF30031D8E
:100370000030D0005108D0040319D4290130A30063
:10038000AC010130AD007F202130DB00FF30DA000E
:10039000DB0BCB29CE29DA0BCB29C8296030DA0058
:1003A000DA0BD02900000000031383160130A800E7
:1003B0002F215008013A031DDF296621E22923304D
:1003C000AA00A020A0308B00031383162108003A56
:1003D000FF3003190030D1002008003AFF30031D20
:1003E0000030D0005008D1055108003A0319372ACF
:1003F0002130AA00A020A101013083120505D100FF
:100400005108003AFF30031D0030D200003085183B
:100410000130D1005108003AFF30031D0030D000F8
:100420005008D204003005190130D1005108003ABB
:10043000FF30031D0030D00050085204D100510895
:10044000003A0319252A0000FC295B30DB00FF304D
:10045000DA00DB0B2C2A2F2ADA0B2C2A292AAB30C4
:10046000DA00DA0B312A0000073081008B16031303
:1004700083122008013AFF30031D0030D10021080B
:10048000003AFF30031D0030D0005008D10551085C
:10049000003A0319882A6621A0010130831205055C
:1004A000D1005108003AFF30031D0030D200003067
:1004B00085180130D1005108003AFF30031D00308B
:1004C000D0005008D204003005190130D100510885
:1004D000003AFF30031D0030D00050085204D10014
:1004E0005108003A0319762A00004D2A5B30DB00E0
:1004F000FF30DA00DB0B7D2A802ADA0B7D2A7A2A8C
:10050000AB30DA00DA0B822A0000073081008B164C
:10051000E429892AFF3FFF3FFF3FFF3FFF3FFF3FA7
:02400E00C43FAD
:00000001FF
